:020000040000FA
:0600000026EF02F01200E1
:0600080002EF05F01200FA
:0600180003EF04F01200EA
:06002A000200900400003A
:10003000000100003300000086040000DF00000023
:040040000A000000B2
:0C0044000000002824C46C0000002810FC
:10005000001000047C00428418E43C806C600000C6
:10006000102800404C7EFE7CFEFEFE7CFE0004FE5E
:10007000FEFEFE7CFE7CFE6280FCF8FCC6E0860094
:10008000400020020004FE1C0C1C0012FE000400B4
:10009000003E3E1C3E103E12203C383C22202200F6
:1000A000008220A80000E0FE54C892A03882101000
:1000B0000A1006088A42868228A2528E92926C6AA0
:1000C00028288280928892828292908210820210E6
:1000D00002402082908290928002040228108AFEC0
:1000E00020824002802A1222122A102A100002FEC8
:1000F000822010222828102A20020402141226101E
:100100000082406800F20028FE10AAC044447C7CB3
:100110000C10061092FE8AA248A2929092926C6CE9
:100120004428448A9E8892828292909210FE82286D
:1001300002301082908A9892FE02020C100E928277
:1001400010828002402A1222122A7E2A105E0208A1
:10015000FE1C20222828202AFC02020C080C2A6CF3
:10016000EE6C403E0000E0FE542644008238101041
:1001700000100020A20292D2FEA292A0929400004F
:100180008228289082889282449290921082FC4425
:100190000240088290849492800204022810A28275
:1001A00008FE4002202A1222122A902A1000BC14B3
:1001B000022020222828202A22020402141032823F
:1001C000001040680000002848460A00000028107F
:1001D000001000407C00628C089C0CC06C78000011
:1001E000002810607C7E6C443882805EFE00808235
:1001F00002FEFE7C607A628C80FCF8FCC6E0C200E5
:1002000004002002001E0C22FE1A403C0E000022B8
:10021000003E1E1C103E1024243C383C222022822A
:04022000000080A8B2
:0C02240092688068936A81689468826820
:10023000956A836A9668846812002A0EC06E0B0E57
:10024000C16E2A0EC06E0B0EC16EC280C280C29AF1
:10025000C2981200D9CFE6FFE1CFD9FF2A0EC06EB7
:100260000B0EC16EC280C282C2B2FED7E552E7CF8A
:10027000D9FF120012000001080EA06F070EA16F37
:10028000A007000EA15BA051A111FAE11200D9CF85
:10029000E6FFE1CFD9FF936AFD0EDB50816E8394B8
:1002A000EADF8384E8DF83949368E552E7CFD9FFE0
:1002B0001200D9CFE6FFE1CFD9FF936AFD0EDB50E4
:1002C000816E8090D8DF8080D6DF80909368E55281
:0602D000E7CFD9FF120088
:0A02D6002A0EF66E000EF76E000E01
:1002E000F86E00010900F550DA6F0900F550DB6F78
:1002F00003E1DA6701D03DD00900F550D56F090060
:10030000F550D66F0900F550D76F09000900F55078
:10031000E96E0900F550EA6E090009000900F55080
:10032000D86F0900F550D96F09000900F6CFDCF04D
:10033000F7CFDDF0F8CFDEF0D5C0F6FFD6C0F7FF7F
:10034000D7C0F8FF0001D85302E1D95307E00900F4
:10035000F550EE6ED807F8E2D907F9D7DCC0F6FF02
:10036000DDC0F7FFDEC0F8FF0001DA07000EDB5B3F
:04037000BFD71200E1
:0C037400D9CFE6FFDACFE6FFE1CFD9FFDA
:10038000E2CFDAFFAC6AAB6AFD0EDBB0AC88DBA271
:1003900002D0AC8CAB8CDBB4AC8EDBA602D0AB88CD
:1003A00001D0AB8ADBB8AC849E98DBBAAB86DBAC01
:1003B00002D09D8A01D09D9A9E9ADBAE02D09D8884
:1003C00001D09D98FB0EDB50AF6EFB0EFC0EDBCF19
:1003D00001F001C000F0016A0050B06EAC8AAB8E33
:1003E000949C948EAC50100B04E0AC50800B01E157
:0E03F000948CE552E5CFDAFFE7CFD9FF12007B
:0203FE00D9CF55
:10040000E6FFDACFE6FFE1CFD9FFE2CFDAFFACAC0F
:1004100004D0AC900001E9B3AC80FD0EDB50AD6EB2
:0C042000E552E5CFDAFFE7CFD9FF12006C
:04042C00000EF36E5D
:1004300000EE00F0040E01D81200EA6002D0EE6A6D
:0C044000FCD7F350E9601200EE6AFCD714
:04044C0013EE00F0BB
:1004500023EE00F0F86A059C6BEC01F042EC02F030
:080460008CEC05F0FBD7120043
:08046800FE0EE3CFE9FFFF0ED9
:10047000E3CFEAFFF36AF46AEE5203E0F34AF42AA8
:04048000FBD7120094
:02048400120064
:0A048600000000000000000000006C
:1004900000000000000000000000002D2D2D2D2D7B
:1004A0002D010000004643414C4C424F583320443C
:1004B0004953504C4159203578372056312E303031
:0304C0000A0D0022
:0608000026EF02F01200D9
:0A080600DACFE4FFE2CFDAFFE6529A
:10081000E552E5CFDAFF1100DACFE4FFE2CFDAFFED
:10082000E9CFE4FFEACFE4FFF6CFE4FFF7CFE4FF40
:10083000F5CFE4FFF3CFE4FFF4CFE4FFFACFE4FF1A
:1008400000EE04F0020EE80403E3EECFE4FFFBD772
:1008500000EE00F0040EE80403E3EECFE4FFFBD764
:10086000E652F2A4ABD0F294FA0ED76E5A0ED66EC0
:100870000101062B000E0723082B0923040E08197B
:1008800001E1095147E1086B096B125127E092D948
:100890008DD988D983D97ED90001A26B080EA25DBB
:1008A00012E201011351132BEA6AAD0FE96E000E3B
:1008B000EA22EF50E66EA3C0E6FF8CD9E552E5527E
:1008C0000001A22BEBD7A32B060EA35D01E1A36BC6
:1008D00001011351280801E2136B1CD00001A26B27
:1008E000080EA25D12E2070ED880A255EA6AA40F94
:1008F000E96E000EEA22EF50E66EA3C0E6FF6AD969
:10090000E552E5520001A22BEBD7A32B050EA35D08
:1009100001E1A36B0101D890075104E6E80E065DE2
:10092000030E07594BE3115149E1066B076B102B7E
:100930001051390833E2300E106F0F2B0F5135086C
:100940002DE2300E0F6F0E2B0E51390827E2300EBC
:100950000E6F0D2B0D51350821E2300E0D6F0C2B53
:100960000B5D08E10C51390805E2310E0B6F300EBA
:100970000C6F14D0310E0B5D08E10C51390805E203
:10098000320E0B6F300E0C6F09D0320E0B5D06E18C
:100990000C51330803E2300E0B6F0C6F10C1ABF03B
:1009A0000FC1AAF000013A0EA96F0EC1A8F00DC147
:1009B000A7F0A66F0CC1A5F00BC1A4F0E55200EEA4
:1009C00003F0040EE80403E3E5CFEDFFFBD700EEF0
:1009D00005F0020EE80403E3E5CFEDFFFBD7E5CF1A
:1009E000FAFFE5CFF4FFE5CFF3FFE5CFF5FFE5CF65
:1009F000F7FFE5CFF6FFE5CFEAFFE5CFE9FFE5CF6B
:100A0000DAFF1100D8CFE4FFE0CFE4FFE46EDACFE5
:100A1000E4FFE2CFDAFFE9CFE4FFEACFE4FFF6CF6D
:100A2000E4FFF7CFE4FFF5CFE4FFF3CFE4FFF4CF2B
:100A3000E4FFFACFE4FF00EE04F0020EE80403E363
:100A4000EECFE4FFFBD700EE00F0040EE80403E372
:100A5000EECFE4FFFBD7E652D9CFE6FFE1CFD9FFD7
:100A6000020EE1269E50200B24E09D50200B21E039
:100A7000AB50040B01E0010EE76E010EE7CFDBFF88
:100A8000AE50DF6E010EDB5003E1AB50020B0BE00A
:100A9000AB98AE50E86EAB88480EE66EFFEC01F006
:100AA000E552FF0004D0DFCFE6FF01DAE5529E9A5F
:100AB00001D0B2DE020EE15C02E2E16AE552E16ED3
:100AC000E552E7CFD9FFE55200EE03F0040EE8044B
:100AD00003E3E5CFEDFFFBD700EE05F0020EE804DF
:100AE00003E3E5CFEDFFFBD7E5CFFAFFE5CFF4FF5A
:100AF000E5CFF3FFE5CFF5FFE5CFF7FFE5CFF6FF55
:100B0000E5CFEAFFE5CFE9FFE5CFDAFFE550E5CF36
:100B1000E0FFE5CFD8FF100038D8200EF26E840E2B
:100B2000F16ED08ED768D66A820ED56EF28E000135
:100B3000200EA46FA56F570EA66F410EA76F490E2A
:100B4000A86F540EA96F200EAA6FAB6F25D828D8B6
:100B50002BD82ED831D834D82DD828D823D81ED881
:100B600019D82CD8180EE66EE66A5C0EE66EBAEC62
:100B700001F0E552E552E5529D8A9F8A9D989F8833
:100B8000AC8AF28EF28CFFD712000F0EC11212EF58
:100B900001F01200838C1200839C120081801200ED
:100BA00081901200818212008192120081841200D1
:100BB00081941200818612008196120081881200B1
:100BC00081981200838A1200839A1200838812008F
:100BD00083981200D9CFE6FFE1CFD9FF020EE126BC
:100BE000FE0EDB50040A21E0070A19E0010A11E0B9
:100BF000030A09E0010A01E01ED0DCDFD9DFD4DFFF
:100C0000CFDFCADF18D0D2DFD7DFCEDFC9DFC4DF46
:100C100012D0C8DFD1DFCCDFC3DFBEDF0CD0BEDF38
:100C2000CBDFC6DFC1DFB8DF06D0B4DFC5DFC0DF92
:100C3000BBDFB6DF00D00101125105E0FD0EDB5035
:100C4000DE6EDD6A6CD0FE0EDB50040A55E0070A4A
:100C500040E0010A2BE0030A16E0010A01E05FD040
:100C6000FD0EDB50E00FF76A440FF66E000EF72220
:100C70000800F5CF00F0016A00BE016800C0DEFF89
:100C800001C0DDFF4CD0FD0EDB50E00FF76AA40F72
:100C9000F66E000EF7220800F5CF00F0016A00BEE4
:100CA000016800C0DEFF01C0DDFF39D0FD0EDB5062
:100CB000E00FF76A040FF66E010EF7220800F5CF79
:100CC00000F0016A00BE016800C0DEFF01C0DDFF68
:100CD00026D0FD0EDB50E00FF76A640FF66E010EB2
:100CE000F7220800F5CF00F0016A00BE016800C0DD
:100CF000DEFF01C0DDFF13D0FD0EDB50E00FF76A11
:100D0000C40FF66E010EF7220800F5CF00F0016A5D
:100D100000BE016800C0DEFF01C0DDFF00D0DECFF5
:100D200000F0DDCF01F0020E0016000E0116D89083
:100D3000015004E6010E005C000E015802E348DF9A
:100D400001D044DF41DF3EDFDECF00F0DDCF01F038
:100D5000040E0016000E0116D890015004E6010E94
:100D6000005C000E015802E333DF01D02FDF2CDFDF
:100D700029DFDECF00F0DDCF01F0080E0016000EF7
:100D80000116D890015004E6010E005C000E0158D7
:100D900002E31EDF01D01ADF17DF14DFDECF00F021
:100DA000DDCF01F0100E0016000E0116D890015094
:100DB00004E6010E005C000E015802E309DF01D0D9
:100DC00005DF02DFFFDEDECF00F0DDCF01F0200E19
:100DD0000016000E0116D890015004E6010E005CCA
:100DE000000E015802E3F4DE01D0F0DEEDDEEADEB3
:100DF000DECF00F0DDCF01F0400E0016000E011630
:100E0000D890015004E6010E005C000E015802E388
:100E1000DFDE01D0DBDED8DED5DEDECF00F0DDCFD9
:100E200001F0800E0016000E0116D890015004E665
:100E3000010E005C000E015802E3CADE01D0C6DEDE
:100E4000C3DEC0DEFE0EDB50040A21E0070A19E013
:100E5000010A11E0030A09E0010A01E01ED0ACDE3C
:100E6000A5DEA0DE9BDE96DE18D0A2DEA3DE9ADE33
:100E700095DE90DE12D098DE9DDE98DE8FDE8ADE73
:100E80000CD08EDE97DE92DE8DDE84DE06D084DE30
:100E900091DE8CDE87DE82DE00D0020EE15C02E2B3
:100EA000E16AE552E16EE552E7CFD9FF1200D9CFF2
:100EB000E6FFE1CFD9FFAECFACF09EAAFED7AECF12
:100EC0000AF10001AC51160A01E19AD0030A01E1CE
:100ED00095D0010A01E188D0070A72E0010A5EE0BC
:100EE000030A55E0010A4CE01F0A47E0010A42E00C
:100EF000030A3DE0010A38E0070A33E0010A2EE068
:100F0000030A29E0010A24E00F0A1FE0010A1AE09F
:100F1000030A15E0010A10E0070A0BE0010A06E0E7
:100F2000030A01E075D00AC1A4F072D00AC1A5F08D
:100F30006FD00AC1A6F06CD00AC1A7F069D00AC16F
:100F4000A8F066D00AC1A9F063D00AC1AAF060D0A7
:100F50000AC1ABF05DD00AC10BF15AD00AC10CF145
:100F600057D00AC10DF154D00AC10EF151D00AC1B7
:100F70000FF14ED00AC110F14BD00AC111F148D087
:100F80000AC112F10101136B0001A36B41D00101F1
:100F9000146B0101136B0001A36B3AD001011451D2
:100FA000142BEA6AAD0FE96E000EEA220AC1EFFFC8
:100FB00001011451270803E20101270E146F28D004
:100FC0000101146B270E0101145D0BE201011451A4
:100FD000EA6AAD0FE96E000EEA22EF6A0101142BF6
:100FE000F1D70101146B14D0EB0E01010A5D05E18C
:100FF000310EE66EFFEC01F0E5520AD0FF0008D09A
:10100000150EE66E010EE66E07D8E552E55200D0E9
:10101000E552E7CFD9FF1200D9CFE6FFE1CFD9FFE4
:10102000020EE126DE6ADD6ADE6ADD6ADECF00F0EE
:10103000DDCF01F000C0E6FF01C0E6FFFD0EDBCF13
:10104000E6FFFE0EDBCFE6FF34EC02F0E552E552A0
:10105000E552E7CF01F0E552E7CF00F0F3CF02F021
:10106000F4CF03F001500318E8AE02D0033404D0EB
:101070000250005C0350015828E2ACA2FED7FD0EDE
:10108000DBCF00F0FE0EDBCF01F0DE500024E96E76
:10109000DD500120EA6EEF50E66EFFEC01F0E55204
:1010A0000101046B056B960E05AF02D0D89003D0FA
:1010B000045D000E055904E2042B000E0523F3D74E
:1010C000DF2A010E01E3DB2AB1D7020EE15C02E266
:0E10D000E16AE552E16EE552E7CFD9FF12006A
:020000040030CA
:0100000025DA
:010001000EF0
:010002003FBE
:0100030000FC
:010005008179
:010006008079
:010008000FE8
:01000900C036
:01000A000FE6
:01000B00E014
:01000C000FE4
:01000D0040B2
:00000001FF
